:100000000C942A000C9447000C9447000C94470071
:100010000C9447000C9447000C9447000C94470044
:100020000C9447000C9447000C9447000C94470034
:100030000C9447000C946D000C9447000C944700FE
:100040000C9447000C9447000C9447000C94470014
:100050000C94470011241FBECFE5D8E0DEBFCDBF12
:1000600010E0A0E6B0E0E6E9F7E002C005900D92EE
:10007000A236B107D9F711E0A2E6B0E001C01D92A7
:10008000A432B107E1F70E9493000C94C9030C94C9
:100090000000DF93CF9300D0CDB7DEB79C011A826A
:1000A000198240EA5FE008C0CA010197F1F789812F
:1000B0009A8101969A83898389819A8128173907C1
:1000C0009CF70F900F90CF91DF91089590BD89B963
:1000D000549A579A8EE880BD08951F920F920FB6DA
:1000E0000F9211248F93EF93FF938FEF8093600013
:1000F000E0916200F0E08CB1ED59FF4F8083809178
:1001000062008F3B30F4809162008F5F80936200C9
:1001100002C010926200FF91EF918F910F900FBE7D
:100120000F901F9018958FEF8ABB87BB84BB98EF09
:1001300091BB97E092BB8BBB88BB85BB819902C00A
:1001400042E001C041E0829B43E0819902C0829B72
:1001500044E010BC87E689B9549A579A8EE880BD6E
:10016000789421E031E060EA7FE05FEFE5E38091A1
:100170006000882331F0809160008150809360009E
:1001800002C0109262009698413009F0B8C0313038
:1001900009F059C0213049F48091630085BB8091FA
:1001A0006B0088BB80917300D9C2223049F48091E2
:1001B000640085BB80916C0088BB80917400CEC2C6
:1001C000233049F48091650085BB80916D0088BB28
:1001D00080917500C3C2243049F48091660085BBCC
:1001E00080916E0088BB80917600B8C2253049F4BA
:1001F0008091670085BB80916F0088BB80917700FC
:10020000ADC2263049F48091680085BB80917000B2
:1002100088BB80917800A2C2273049F480916900A0
:1002200085BB8091710088BB8091790097C228308E
:1002300009F095C280916A0085BB8091720088BBED
:1002400080917A008BC2323009F089C2213049F4A2
:1002500080917B0085BB8091830088BB80918B005F
:100260007DC2223049F480917C0085BB809184005E
:1002700088BB80918C0072C2233049F480917D004C
:1002800085BB8091850088BB80918D0067C224303A
:1002900049F480917E0085BB8091860088BB809167
:1002A0008E005CC2253049F480917F0085BB80912F
:1002B000870088BB80918F0051C2263049F480911D
:1002C000800085BB8091880088BB8091900046C2E9
:1002D000273049F48091810085BB8091890088BBDB
:1002E000809191003BC2283009F039C28091820090
:1002F00085BB80918A0088BB809192002FC24230DA
:1003000009F0B8C0313009F059C0213049F480916A
:10031000930085BB80919B0088BB8091A3001EC287
:10032000223049F48091940085BB80919C0088BB69
:100330008091A40013C2233049F48091950085BBBD
:1003400080919D0088BB8091A50008C2243049F4AB
:100350008091960085BB80919E0088BB8091A6000D
:10036000FDC1253049F48091970085BB80919F00A5
:1003700088BB8091A700F2C1263049F48091980093
:1003800085BB8091A00088BB8091A800E7C1273081
:1003900049F48091990085BB8091A10088BB809130
:1003A000A900DCC1283009F0DAC180919A0085BB30
:1003B0008091A20088BB8091AA00D0C1323009F0A0
:1003C000CEC1213049F48091AB0085BB8091B30050
:1003D00088BB8091BB00C2C1223049F48091AC003F
:1003E00085BB8091B40088BB8091BC00B7C123302D
:1003F00049F48091AD0085BB8091B50088BB8091A8
:10040000BD00ACC1243049F48091AE0085BB809121
:10041000B60088BB8091BE00A1C1253049F480910F
:10042000AF0085BB8091B70088BB8091BF0096C1AB
:10043000263049F48091B00085BB8091B80088BB1C
:100440008091C0008BC1273049F48091B10085BBF9
:100450008091B90088BB8091C10080C1283009F02B
:100460007EC18091B20085BB8091BA0088BB80912B
:10047000C20074C1433009F0B8C0313009F059C02E
:10048000213049F48091C30085BB8091CB0088BBAB
:100490008091D30063C1223049F48091C40085BBB0
:1004A0008091CC0088BB8091D40058C1233049F49E
:1004B0008091C50085BB8091CD0088BB8091D5001F
:1004C0004DC1243049F48091C60085BB8091CE0097
:1004D00088BB8091D60042C1253049F48091C70085
:1004E00085BB8091CF0088BB8091D70037C1263073
:1004F00049F48091C80085BB8091D00088BB809171
:10050000D8002CC1273049F48091C90085BB809167
:10051000D10088BB8091D90021C1283009F01FC1CA
:100520008091CA0085BB8091D20088BB8091DA009F
:1005300015C1323009F013C1213049F48091DB003C
:1005400085BB8091E30088BB8091EB0007C122301E
:1005500049F48091DC0085BB8091E40088BB8091E8
:10056000EC00FCC0233049F48091DD0085BB809114
:10057000E50088BB8091ED00F1C0243049F4809102
:10058000DE0085BB8091E60088BB8091EE00E6C06E
:10059000253049F48091DF0085BB8091E70088BB5E
:1005A0008091EF00DBC0263049F48091E00085BBEC
:1005B0008091E80088BB8091F000D0C0273049F4DA
:1005C0008091E10085BB8091E90088BB8091F100BA
:1005D000C5C0283009F0C3C08091E20085BB80917E
:1005E000EA0088BB8091F200B9C0443009F0B7C07E
:1005F000313009F059C0213049F48091F30085BBB6
:100600008091FB0088BB80910301A8C0223049F48F
:100610008091F40085BB8091FC0088BB809104012F
:100620009DC0233049F48091F50085BB8091FD0089
:1006300088BB8091050192C0243049F48091F60076
:1006400085BB8091FE0088BB8091060187C0253064
:1006500049F48091F70085BB8091FF0088BB8091B1
:1006600007017CC0263049F48091F80085BB809159
:10067000000188BB8091080171C0273049F4809146
:10068000F90085BB8091010188BB8091090166C09A
:10069000283009F064C08091FA0085BB8091020186
:1006A00088BB80910A015AC0323009F058C021300D
:1006B00049F480910B0185BB8091130188BB809127
:1006C0001B014CC0223049F480910C0185BB809104
:1006D000140188BB80911C0141C0233049F48091F2
:1006E0000D0185BB8091150188BB80911D0136C02D
:1006F000243049F480910E0185BB8091160188BB9E
:1007000080911E012BC0253049F480910F0185BBDB
:100710008091170188BB80911F0120C0263049F4C9
:100720008091100185BB8091180188BB80912001C8
:1007300015C0273049F48091110185BB80911901C2
:1007400088BB809121010AC0283049F480911201B0
:1007500085BB80911A0188BB809122018BBBCB01A4
:100760000197F1F72F5F5BBB58BB55BB293058F0A1
:100770003F5F333008F031E0969A8E2F8A95F1F77B
:10078000969821E0F4CC979A8E2F8A95F1F7979856
:06079000EECCF894FFCF4F
:02079600010060
:00000001FF
